:100000004D298030A100FE30AF200130AF20753087
:10001000AA0030300229A101A117B200B208031DC5
:100020001328030114280130B2020310A20CA20C01
:10003000A20CC0302205403EB207FE30AF2032088D
:10004000AF28A101A117B200FE30AF203208AF28BF
:10005000A401AD00AE01A01124080319A0150530BC
:10006000A3002730AC00103041200330AC00E83052
:100070004120AC0164304120AC010A3041202D0800
:100080004828AB002E08AA002D08A900162129082F
:10009000A900A3030319A01124080319522823025D
:1000A000031859282908031DA011A0195928303E0A
:1000B000AF280800A3002408031948292308AF200B
:1000C000A4035B28B0000611861183160611861161
:1000D0000F30860583123008A0188C283E30AA0005
:1000E000803002213330AF00A0201330AA008830C6
:1000F0000221A02064300121A0206430012122309F
:10010000AF00A02028308B200C308B2006308B20B5
:10011000A01430088C282014AF00201C9A288611C7
:10012000033C031C9F289F200530AA00DC300221DD
:10013000031408002014FE3C0319AD288615201C6A
:10014000201006150F3086052F08F0398604061199
:10015000AF0E2018A0283230012130084829A11BF9
:100160006228AC00220884002509841780058413C6
:10017000AC080319D928F030AE002B088038AD0048
:10018000F030AE030319AE000319AC030319D928EC
:10019000C928E420030126182508AB1F2508AB0851
:1001A00003190301AD0FD6288006BD28D72800000B
:1001B000C028250884178004482983178001840AF1
:1001C000FF3E031DDE284829270826040319A60A36
:1001D0008030261AA7062619A706A618A706270DF7
:1001E000A60DA70D26084829AC01AB00FF30AB07D0
:1001F000031CAC07031C48290330AA00DF3002218E
:10020000F628AA01E83EA900AA09FC30031C0B2924
:10021000A90703180829A9070000AA0F0829291807
:100220001129A91C1529000015290800AE01AD01EE
:100230001030AF002A0DAD0DAE0D2B08AD022C080D
:10024000031C2C0FAE0203182C292B08AD072C0819
:1002500003182C0FAE070310A90DAA0DAF0B1A2916
:10026000290848291030B300AA01A901B00CAF0C2D
:10027000031C40292B08A9072C0803182C0FAA07D8
:10028000AA0CA90CAE0CAD0CB30B36292D084829CD
:1002900083138312031300000800A00107309F009E
:1002A000B13083168500FF30860081132030840032
:1002B00060308312DE20A03084005030DE202030F9
:1002C00084003030DD20C830F4200120533062201B
:1002D00069306220673062206E30622061306220B7
:1002E00062206C306220203062207A3062206F30D1
:1002F0006220653062206B306220653062206E3093
:10030000622039140D2AC5013F03A800C90149081C
:100310002802031C9C29BF21B91C9A294508A90061
:100320004908A200A901A20A0314A90DA20B95294C
:100330002908C504C90F8729B5014508B400B50CC3
:10034000B40CB50CB40CB50CB40CB50CB40C0F302B
:10035000B5053508B0003408AF00AC010A30AB0079
:100360003221B4002E08B500B7014508B6000F30A1
:10037000B6050030B70534083607C5000800BD01D2
:10038000BC010618D4290130F420BC0A0319BD0AA7
:100390000B303D02031CD329031DD229B9303C0286
:1003A000031CD329B22CC1299B30F4200618B914A0
:1003B000061CB910391CFF29B5014608B400B70165
:1003C0003C30B6000430A9000310B70CB60CA90BE2
:1003D000E429B60A0319B70A3508AA003408A900A7
:1003E0003708AC003608AB001621C0008030A100F1
:1003F0000230A20040080D20FF306220072A803022
:10040000A1008E3021200230A40046082920C60A0F
:1004100005151E30F42005110800BE01C601391172
:100420003919B12ABD01BC01061C272ABC0A0319CF
:10043000BD0A0130F420AF303D02031C262A031D03
:10044000252AC9303C02031C262AB22C142ABD01DD
:10045000BC0106185B2ABC0A0319BD0A0A30F42045
:1004600039184F2A3C08613A3D04031D412A803067
:10047000A1008E30212035306220393062200515F0
:100480004E2A3C08643A3D04031D482A05114E2AB1
:100490003C08FA3A3D04031D4E2AB22C5A2A113068
:1004A0003D02031C5A2A031D592A95303C02031CA5
:1004B0005A2AB22C292A3D303E02031C602AB22C53
:1004C000BE0A3D08031D682A65303C02031C692AE8
:1004D0003915391CB02AB5013E08B400B7013D30CA
:1004E000B6000430A9000310B70CB60CA90B732A90
:1004F000B60A0319B70A3508AA003408A900370854
:10050000AC003608AB001621C0008030A10080305E
:1005100021205330622069306220673062206E30C3
:1005200062206130622062206C30622020306220C4
:100530006730622065306220763062206F30622042
:100540006E30622064306220653062206E3062203E
:100550008030A1000230A20040080D20FF30622050
:10056000102A391CDB2A0120493062206E306220BB
:10057000693062207430622069306220613062200C
:100580006C306220693062207330622065306220F6
:1005900072306220653062206E3062202E30622020
:1005A000622062208030A100C03021200E30A400E3
:1005B0005F305A20092B0930C0000130A2004008EA
:1005C0000B20A1010A3047020318E82A20306220DC
:1005D0008030A100470828203A3062200230A40071
:1005E000440829203A3062203030622062204408DA
:1005F000031DFB2A822C1E30440203190130031D07
:100600000301B80003018618013038050319092BCE
:10061000822C391D802CC9010F3049020318132B7D
:10062000BF21C90F0C2BBF21BF21BF21B91C1A2B21
:1006300085151B2B85111230C9001430490203188F
:10064000242BBF21C90F1D2BBF210730BF008321E1
:100650004508C400BF210630BF0083214508C700FC
:10066000BF210630BF0083214508C1000330BF0011
:1006700083214508C8000530BF0083214508C30019
:100680000830BF0083214508C200BF21391C4A2B16
:10069000391001208030A100803021200830A400D2
:1006A00020305A208030A100C03021201030A4001A
:1006B00020305A2080302120A10101304802031D42
:1006C000662B4D306220613062209B2B0230480245
:1006D000031D6F2B44306220693062209B2B033056
:1006E0004802031D782B573062206F3062209B2B0D
:1006F00004304802031D812B443062206F30622099
:100700009B2B05304802031D8A2B56306220723025
:1007100062209B2B06304802031D932B5A30622027
:10072000613062209B2B07304802031D9B2B5A30FF
:1007300062206F3062208030A100C030212041084B
:1007400028202030622001304302031DB62B4A309E
:100750006220613062206E3062207530622061302C
:1007600062207230622069306220752C02304302B0
:10077000031DCB2B46306220653062206230622040
:1007800072306220753062206130622072306220E7
:1007900069306220752C03304302031DD92B4D3084
:1007A00062206130622062207230622074306220E8
:1007B000752C04304302031DE82B41306220703059
:1007C000622072306220693062206C306220752CA9
:1007D00005304302031DF32B4D306220653062204B
:1007E00069306220752C06304302031D002C4A300C
:1007F0006220753062206E30622069306220752C74
:1008000007304302031D0D2C4A30622075306220F0
:100810006C30622069306220752C08304302031D61
:10082000222C4130622075306220673062207530A2
:100830006220733062207430622075306220733021
:100840006220752C09304302031D392C533062207D
:100850006530622070306220743062206530622022
:100860006D3062206230622065306220723062201A
:10087000752C0A304302031D4C2C4F3062206B3024
:100880006220743062206F306220623062206530F6
:10089000622072306220752C0B304302031D612CE4
:1008A0004E3062206F3062207630622065306220E8
:1008B0006D306220623062206530622072306220CA
:1008C000752C0C304302031D752C443062206530BA
:1008D000622063306220653062206D3062206230B9
:1008E0006220653062207230622020306220273022
:1008F00062208030A1000230A40042082920812C0F
:10090000B22C0D2A0F30C0008514C6010F304602EC
:100910000318B12C0530A2004030A5007F30AB0099
:100920001430B1208030A1000130A20040080D2019
:100930000230A4004608292005150530A2004030E9
:10094000A5007F30AB000230B120851005110530C5
:10095000A2004030A5007F30AB003A30B120C60F76
:10096000862C132B012047306220653062206220E4
:100970006E30622020306220733062206930622045
:10098000673062206E3062206130622062206C30FD
:100990006220203084006030DE20A030840050309F
:1009A000DE20203084003030DD200618B915061C0A
:1009B000B91103010618013EB919013C031DE62CCB
:1009C000BA0A0319BB0A0130F420D92C0301B91962
:1009D0000130013A0319B911031DB91503010618B5
:1009E000013EB919013C031DFB2CBA0A0319BB0ACD
:1009F0000130F420EE2C03303B02DE3003193A02C2
:080A00000318C92C39140D2A5A
:02400E00503F21
:00000001FF
